:08000800FF00030E8301A100BB
:100010007F08A0000A08A8008A01A00E0408A20018
:100020007708A3007808A4007908A5007A08A6003C
:100030007B08A700831383128C308400001C2228C5
:100040000C183528220884002308F7002408F8003B
:100050002508F9002608FA002708FB0028088A006E
:10006000210E8300FF0E7F0E09008A1141280A101D
:100070008A100A11820748344F34523441343A34DA
:1000800000340030BD02031C0130BE020130031CED
:100090000230BF020030031C0130C002C008031D43
:1000A00064283F08003C031C64284030BD074230F0
:1000B00003184330BE070F3003181030BF0700305D
:1000C00003180130C007C10A41083C3C031DAB289E
:1000D000C60AC10146083C3C031DAB28C50AC6013F
:1000E0004508183C031DAB28C40AC50144081D3C43
:1000F000031D83284308023C031D8328420803395B
:10010000003A031DA32844081E3C031D8B28430806
:10011000023C0319A32844081F3C031D9F284308E1
:10012000043C0319A3284308063C0319A3284308E9
:10013000093C0319A32843080B3C0319A3284408CE
:10014000203C031DA528C30AC40143080D3C031D20
:10015000AB28C20AC3010C108A112228C0010F303B
:10016000BF004230BE004030BD0085309000831695
:100170000C1483128A11222A5730840000080319B4
:10018000D0280130F800F701F70BC428F80BC3287A
:100190004A30F700F70BCA2800000000800BC12886
:1001A000003405114230F700F70BD428000042302C
:1001B000F700F70BD928000005154230F700F70BC0
:1001C000DF2800004230F700F70BE428000000347D
:1001D000851456088600D1200130D700BC20003499
:1001E0004708840055088000840A8001C70A00344B
:0201FE000030CF
:100200008A000E2A0000F701F8015508031056185D
:10021000F707F70CF80CD618F707F70CF80C561977
:10022000F707F70CF80CD619F707F70CF80C561A65
:10023000F707F70CF80CD61AF707F70CF80C561B53
:10024000F707F70CF80CD61BF707F70CF80C8A1118
:100250003729851002308600D1204230F700F70B95
:100260002F2900005308D5002830D6000329540850
:100270007807D300D40153085402031849291430D5
:100280008600D1204230F700F70B44290000D40A41
:100290003B290034D4015308540784008008031913
:1002A0005A295308540784000008D500D600E820D6
:1002B000D40A4B2900343030C900CA003A30CB0090
:1002C0003030CC00CD003A30CE003030CF00D000FE
:1002D000D101D201851005150130D700BC2038307E
:1002E0008600D12001308600D12003308600D12045
:1002F0000F308600D120851005150130D700BC20B5
:1003000001308600D1200F308600D120D301530860
:100310003720003803199029D30AD600E82087290E
:100320000130D300D40129214930D3004A218A1158
:100330002D2A5608F80155020318A1295508F7007F
:10034000AD29F7010830D700D50DF70D5608770213
:100350000318F700F80DD70BA429003478085308C8
:10036000D5006430D60099217708D3007808303062
:10037000031DC1295418C729D419C729541A20307C
:10038000C329D4115412F8077808D500F020530877
:10039000D5000A30D60099217708D300780830308C
:1003A000031DD629D419DA29541A2030F807780801
:1003B000D500F0203030D3075308D500F0200034AA
:1003C0000130D300D40129214930C7004508D300AA
:1003D0000130D400AE214930D3004A210130D3008E
:1003E0000330D40029214930C7004608D30001302A
:1003F000D400AE214930D3004A210130D300063069
:10040000D40029214930C7004108D3000130D4006D
:10041000AE214930D3004A218A11342A84011F3089
:10042000830583161F08C0399F009B010730831284
:100430009F00BC01C101C201C301C401C501C601C5
:10044000C701AE28C0308B048316850183120510C6
:1004500083168601831286015B294808410203192D
:0C046000342A4108C800E0292D2A63005E
:040000008A01FF284A
:00000001FF
